:04000000B601B72965
:100008000800B616B61EB612B6190E28B615472041
:10001800031835280830A3005B20A20DA30B102875
:10002800B61E402065206120B61A35203A202208E5
:100038000310B229B616B61EB61236192828FE398C
:10004800B70036150310B229361A3028A60036161E
:1000580047200318352826084E2003183528B61ED1
:10006800B2294020652036113612B6113A088400AC
:1000780038088417800446283A088400380980051F
:100088008417800508003A20652040206120370841
:10009800B6190138A2000830A300A20D03183A20AF
:1000A800031C402065206120A30B51283A206520BD
:1000B8003A08840038080005FF3E3B0884003909E7
:1000C80043283B08840039083D2864007F20031832
:1000D8006928CE20A8010830A300CF207F2003186C
:1000E800A80AAB1EA801A20CA30B7128AB1AA21375
:1000F800CF20220808003A088400380884178004B2
:10010800841300052B1B3806FF3E0800A4002908AD
:100118000319B229AD21A0002518831724088400EB
:10012800200880008313A40AA9038B280408A600CA
:100138003A088400F030B7050830A7000310031808
:10014800B70AB420A60CA70BA3280000AB1A370CDB
:10015800B420B5210314B4202F08A3002E082D299C
:100168008413AB1FC328000838042B1F38068000EF
:10017800841700083804031C38068000CF280008BC
:100188003804031C38062B1B3806800084173809EE
:100198008005CF2837172B081F39003EA1002A08F1
:1001A8000E3E0318A10A371F3A293713A000023060
:1001B8005E213A29B71329080319B7170430A80094
:1001C800250EEB202508EB20240EEB2024080F3900
:1001D800F63E0318073E0A3EF128A000A8030319BB
:1001E800B71329080319FB28280203180800200858
:1001F800031DB713B71B0800303EAD2901308A0034
:1002080028080739820701340234043408341034CA
:1002180020344034803483178001840AFF3E031D54
:100228001029B22903178D0083168C130C1483121E
:100238000C08B22903178C0083168C130C15553043
:100248008D00AA308D008C148C1828290C11B22925
:10025800A301A200FF30A207031CA307031CB229B5
:100268000330A100E7303A212E29A101FC3EA0006D
:10027800A109031C4529FF300000A00703184029E5
:10028800A0076400A10F3F290800A8000221A001CF
:10029800A101A81DA000A819A1002008B2290310D7
:1002A800A00DA10DFF3E031853292008B229031001
:1002B800A10CA00CFF3E03185B292008B229A1015C
:1002C800A301A20002306B29A20001306B29A8000B
:1002D80023082102031D7229220820020430031872
:1002E8000130031902302805031DFF30B2291030F0
:1002F800A600A501A401210DA40DA50D2208A402A4
:100308002308031C230FA502031891292208A40718
:1003180023080318230FA5070310A00DA10DA60B92
:100328007F292008B2291030A800A101A001A70C3C
:10033800A60C031CA5292208A00723080318230FCD
:10034800A107A10CA00CA50CA40CA80B9B292408A0
:10035800B229840031088A0030088200831303130D
:100368008312640008002030840060308A01102164
:10037800A030840050308A01102110308400603091
:100388008A010F219030840060308A010F21831682
:1003980007309F0099018312980183160230980054
:1003A8008312F701F80183168610061188010710D9
:1003B8008710071187128312D9010130A300F43086
:1003C8008A012D2187120A308A012C2187160130D3
:1003D800A300F4308A012D218A110A12F22F071482
:1003E8000A308A013921071008008A110A120323EA
:1003F8007008A000A1010830A200A3018A017B2196
:10040800E4007008A000A1010830A200A3018A013D
:100418007B212408B2002508B30032088A0149214B
:10042800EF008710B830640788008A01F321403054
:100438006A0788008A01F3218A110A12CE22640011
:100448006608003C8A110A12031D302A63086F04EB
:1004580088008A110A12332A63086F0688008A0105
:10046800F321080087103E3088008A01F3218614A2
:1004780006110130DA00640003305A028A110A12A8
:100488000318812AB830DD006400C0305D028A118B
:100498000A120318712A87108A01F3214030880054
:1004A8008A01F3215D0888008A01F321871401304D
:1004B800DE00640041305E028A110A1203186C2AB9
:1004C80088018A01F321DE0A8A110A12031D5D2AB6
:1004D800DD0A8A110A12031D482A8310861883141C
:1004E80006198614061D861083180615831C061126
:1004F800DA0A8A110A12031D3F2A87108614061188
:100508000130DA00640003305A028A110A12031813
:10051800B12A3E3088008A01F321C03088008A0160
:10052800F321403088008A01F321B83088008A011D
:10053800F3213F3088008A01F32183108618831441
:1005480006198614061D861083180615831C0611C5
:10055800DA0A8A110A12031D862A861406118714DC
:1005680008008A110A1203237008A000A1010830AC
:10057800A200A3018A017B21E400871040306A07AA
:1005880088008A01F321B830640788008A01F321C2
:10059800871408008A110A12032387148316FF3070
:1005A80088008312071507140A308A0139210808C0
:1005B800E30007100A308A01392107140A308A013A
:1005C80039210808E30007100711831688018312F0
:1005D800871040306A0788008A01F321B830640721
:1005E80088008A01F321871408008A01B5228A014C
:1005F800CE226308580488008A01F32108006400A9
:1006080040306B028A110A12031C122B8610061541
:1006180040306B02EA008A110A12162B8614061162
:100628006B08EA0008000130E6008A01F921E601BA
:10063800080088018A01F321EB0A8A01B522080023
:1006480064006B083F3C8A110A12031D4C2B87106B
:1006580083108618831406198614061D86108318BD
:100668000615831C0611403088008A01F3217008A2
:10067800A000A1010830A200A3018A017B21B200D9
:100688002108B300B830320788008A01F3218714A3
:1006980008008A110A1283236808DA0064005A08DD
:1006A80069028A110A12031C692B5A08EB006D08AB
:1006B800F0008A01F9216E08F0008A01F921720818
:1006C800DA078A110A12031C522B6D08DA0064003B
:1006D8005A086E028A110A12031C822B5A08F0006B
:1006E8006808EB008A01F9216908EB008A01F92101
:1006F8007208DA078A110A12031C6B2B08006400BF
:10070800680869028A110A1203188E2B68086902A0
:10071800E807E90264006D086E028A110A120318DC
:10072800992B6D086E02ED07EE0208006708560760
:10073800EB006C085707F0008A01F9216708560298
:10074800EB006C085707F0008A01F9215608670783
:10075800EB006C085702F0008A01F921670856027D
:10076800EB006C085702F0008A01F9216C08560763
:10077800EB0067085707F0008A01F9216C08560258
:10078800EB0057086707F0008A01F92156086C0743
:10079800EB0067085702F0008A01F9216C0856023D
:1007A800EB0067085702F0008A01F9210800871456
:1007B800D0305507B200FF300318013EB3003208AD
:1007C800A6003308A7000330A200A3018A019721DD
:1007D800B2002508B30000303207CE0002304E07C1
:1007E800CF004E08CD0064004D084F028A110A124E
:1007F800031C0A2C4D088A01162188008A01F3215E
:10080800EB0ACD0A8A110A12031DF72B8A01B522B9
:100818008A011D2308007408EB007608F0006400C4
:10082800700875028A110A12031C212C8A01F92109
:10083800F00A8A110A12031D132C740AEB007608B9
:10084800F0006400700875028A110A12031C342C27
:100858008A01F9217208F0078A110A12031C252C53
:1008680008007608F0007408EB0064006B08730257
:100878008A110A12031C472C8A01F921EB0A8A11F2
:100888000A12031D392C7603F0007408EB0064008B
:100898006B0873028A110A12031C5A2C8A01F92167
:1008A8007208EB078A110A12031C4B2C08008A01F4
:1008B800832368086902DF006D086E02E2006400A5
:1008C80062085F028A110A12031CB42C6208A00095
:1008D800A10102308A015621B2002108B3005F0845
:1008E8003202CB003308031CFF3ECC006D08F00039
:1008F8006808EB0064006B0869028A110A12031C7D
:10090800B32C64008A110A12CC1F9C2C6208A00028
:10091800A10102308A015621B2002108B300320831
:10092800CB0733080318013ECC078A110A12AC2CF6
:100938005F086202B200B301031CB3030310B20DD7
:10094800B30D3208CB0733080318013ECC07F00A71
:100958008A01F921EB0A8A110A12031D7E2C08006C
:100968005F08A000A10102308A015621B2002108C7
:10097800B30062083202CB003308031CFF3ECC00F0
:100988006808EB006D08F000640070086E028A11B8
:100998000A12031CFD2C64008A110A12CC1FE62CD3
:1009A8005F08A000A10102308A015621B200210887
:1009B800B3003208CB0733080318013ECC078A116D
:1009C8000A12F62C62085F02B200B301031CB303DB
:1009D8000310B20DB30D3208CB0733080318013EDC
:1009E800CC07EB0A8A01F921F00A8A110A12031DC1
:1009F800C82C0800E7016508EC000310650DB2007B
:100A0800B301B30D3208033CCB003308031C013E8D
:100A1800003CCC00640067086C028A110A12031CAF
:100A2800542D8A019A2364008A110A12CC1F342D8E
:100A38000430A600A7016708A200A3018A01972134
:100A4800B2002508B3000630B2070318B30A32080B
:100A5800CB0733080318013ECC078A110A12512D1F
:100A68006C086702B200B301031CB3030430A6008C
:100A7800A7013208A2003308A3008A019721B20017
:100A88002508B3000A30B2070318B30A3208CB07A7
:100A980033080318013ECC07EC03E70A8A010E2D40
:100AA80008005A083C3E84000008B200FF30A2004B
:100AB800A20A22080F3C8A110A12031C842D8A11EB
:100AC8000A12702532028A110A12031D5C2D2208AF
:100AD800F1008A110A12842D05308A002208820743
:100AE80030343134323433343434353436343734C2
:100AF8003834393461346234633464346534663488
:100B08000800E7016508EC000310650DB200B301A9
:100B1800B30D3208033CCB003308031C013E003CF4
:100B2800CC00640067086C028A110A12031CBE2DEF
:100B38008A019A236C086702B200B301031CB3034D
:100B48000430A600A7013208A2003308A3008A01D6
:100B58009721B2002508B3000A30B2070318B30A78
:100B68003208CB0733080318013ECC07EC03E70A29
:100B78008A01952D0800E7016508EC000310650D52
:100B8800B200B301B30D3208033CCB003308031C99
:100B9800013E003CCC00640067086C028A110A120E
:100BA800031CF02D8A019A230430A600A7016708C8
:100BB800A200A3018A019721B2002508B3000630DC
:100BC800B2070318B30A3208CB0733080318013EEB
:100BD800CC07E70A8A01CF2D0800E7016508EC0079
:100BE8000310650DB200B301B30D3208033CCB000E
:100BF8003308031C013E003CCC00640067086C020B
:100C08008A110A12031C2B2E8A019A236C08670288
:100C1800B200B301031CB3030430A600A7013208D5
:100C2800A2003308A3008A019721B2002508B30067
:100C38000A30B2070318B30A3208CB07330803187F
:100C4800013ECC070330EC02E70A8A01012E0800B6
:100C5800580888008A01F321EB0A64006B08403CBD
:100C68008A110A12031D492E861006158710403076
:100C780088008A01F321C03088008A01F321B83046
:100C8800610788008A01F321871464006B08803C9F
:100C98008A110A12031D6B2EE10A64006108083CE0
:100CA8008A110A12031D592EE101EB01861406115F
:100CB8008710403088008A01F321B8306107880026
:100CC8008A01F321C03088008A01F32187140800C3
:100CD8008A0183236808DA0064005A0869028A11C5
:100CE8000A12031C922E6D08DD0064005D086E0276
:100CF8008A110A12031C8C2E5A08EB005D08F000BA
:100D08008A01F9217208DD078A110A12031C792E5B
:100D18007208DA078A110A12031C702E08000730BD
:100D2800BA004030B8002030AA00AB01AE01AF01D4
:100D38000230A9005508A400A5019A30B000B101FD
:100D48008A01DE2008000730BA008030B800203061
:100D5800AA00AB018A0169205D3C8A110A12031DB1
:100D6800AE2E0230A9006930B000B101A5013C30B7
:100D78008A018A20DA01640002305A028A110A12B2
:100D88000318D22E8A0155255A083C3E8400710862
:100D98008000DA0A8A110A12031DBF2E3C08A0003F
:100DA800A10104308A015621B2002108B3003D0890
:100DB8003204D00008000730BA008030B800203074
:100DC800AA00AB018A0169205D3C8A110A12031D41
:100DD800E62E0430A9006930B000B101A5013C300D
:100DE8008A018A20DA01640004305A028A110A1240
:100DF80003180A2F8A0155255A083C3E84007108B9
:100E08008000DA0A8A110A12031DF72E3C08A00096
:100E1800A10104308A015621B2002108B3003D081F
:100E28003204D0003E08A000A10104308A015621F6
:100E3800B2002108B3003F083204D100080007308F
:100E4800BA008030B8002030AA00AB018A016920BE
:100E58005D3C8A110A12031D2A2F0630A900693049
:100E6800B000B101A5013C308A018A20DA01640092
:100E780006305A028A110A1203184E2F8A01552584
:100E88005A083C3E840071088000DA0A8A110A1266
:100E9800031D3B2F3C08A000A10104308A01562104
:100EA800B2002108B3003D083204D0003E08A0007B
:100EB800A10104308A015621B2002108B3003F087D
:100EC8003204D1004008A000A10104308A01562153
:100ED800B2002108B30041083204D20008000730EC
:100EE800BA008030B8002030AA00AB018A0169201E
:100EF8005D3C8A110A12031D7A2F8A016920F100CC
:100F080030307102F2007108D50008000730BA00CD
:100F18008030B8002030AA00AB018A0169205D3C0E
:100F28008A110A12031D912F0830A9006930B000F8
:100F3800B101A5013C308A018A20DA016400083039
:100F48005A028A110A120318B52F8A0155255A0820
:100F58003C3E840071088000DA0A8A110A12031DD7
:100F6800A22F3C08A000A10104308A015621B2003A
:100F78002108B3003D083204E8003E08A000A101A2
:100F880004308A015621B2002108B3003F08320418
:100F9800E9004008A000A10104308A015621B200EE
:100FA8002108B30041083204ED004208A000A10165
:100FB80004308A015621B2002108B30043083204E4
:100FC800EE0008005008D6005108D7005208E50086
:100FD80008005008EB005108F00008008A0136228A
:100FE8000830EB003F30F0008A01B522DA016400D6
:100FF80017305A028A150A1203184D285A08163C47
:101008008A150A12031C2A288A150A120F20D500ED
:101018008A150A122A2808308A005A088207473493
:1010280052344134503448344934433420344434FD
:1010380045344D344F342034423459342034433409
:101048004F344D34503453345934533464005508B4
:10105800203C8A150A12031D44280130DD00640073
:1010680003305D028A150A12031841288A011D23DC
:10107800DD0A8A150A12031D33288A150A12462822
:101088008A01DB238A011D23DA0A8A110A12031D49
:10109800FB2F4030D6002030D7001630E5008A01FB
:1010A800FE248A01BF258A0185250530E5008A01CD
:1010B800FE248A01BF250230E5008A01FE240130A2
:1010C800E5008A01FE24E8017F30E900ED013F30A8
:1010D800EE000230F2008A014D230230E8007D3034
:1010E800E9000230ED003D30EE000130F2008A01E7
:1010F8004D230730BA004030B8002030AA00AB01B9
:10110800AE01AF0152308A019B2065308A019B20D5
:1011180061308A019B2064308A019B2079308A01E2
:101128009B203A308A019B200A308A019B200D308F
:101138008A019B200730BA008030B8002030AA000E
:10114800AB018A0169205D3C8A150A12031DA52896
:101158008A016920F1007108A00063308A016321C7
:10116800B2007108A00043308A016321B40032083C
:1011780034048A150A12031D432B7108A00073302A
:101188008A016321B2007108A00053308A016321EB
:10119800B400320834048A150A12031D4C2B710856
:1011A800A00071308A016321B2007108A00051309B
:1011B8008A016321B400320834048A150A12031D17
:1011C800552B7108A00074308A016321B2007108A0
:1011D800A00054308A016321B400320834048A150F
:1011E8000A12031D5E2B7108A0006C308A0163216E
:1011F800B2007108A0004C308A016321B4003208A3
:1012080034048A150A12031D862B7108A000723057
:101218008A016321B2007108A00052308A0163215B
:10122800B400320834048A150A12031D702B7108A1
:10123800A00062308A016321B2007108A000423028
:101248008A016321B400320834048A150A12031D86
:10125800672B7108A0006B308A016321B200710806
:10126800A0004B308A016321B400320834048A1587
:101278000A12031D9C2B7108A00064308A016321A7
:10128800B2007108A00044308A016321B40032081A
:1012980034048A150A12031D922B7108A0006530C8
:1012A8008A016321B2007108A00045308A016321D8
:1012B800B400320834048A150A12031D902B7108F1
:1012C800A00070308A016321B2007108A00050307C
:1012D8008A016321B400320834048A150A12031DF6
:1012E800A12B7108A00075308A016321B200710832
:1012F800A00055308A016321B400320834048A15ED
:101308000A12031D072C7108A00078308A01632196
:10131800B2007108A00058308A016321B400320875
:1013280034048A150A12031D122C7108A0007930A2
:101338008A016321B2007108A00059308A01632133
:10134800B400320834048A150A12031D212C7108CE
:10135800A00066308A016321B2007108A0004630FF
:101368008A016321B400320834048A150A12031D65
:10137800792B7108A00068308A016321B2007108D6
:10138800A00048308A016321B400320834048A1569
:101398000A12031DAE2B7108A00076308A01632162
:1013A800B2007108A00056308A016321B4003208E7
:1013B80034048A150A12031DDB2B7108A00069305A
:1013C8008A016321B2007108A00049308A016321B3
:1013D800B400320834048A150A12031D8D2B7108D3
:1013E800A0006A308A016321B2007108A0004A3067
:1013F8008A016321B400320834048A150A12031DD5
:101408008D2B7108A0006D308A016321B20071082C
:10141800A0004D308A016321B400320834048A15D3
:101428000A12031D742A7108A0006E308A01632114
:10143800B2007108A0004E308A016321B40032085E
:1014480034048A150A12031D762A7108A0006F3029
:101458008A016321B2007108A0004F308A0163211C
:10146800B400320834048A150A12031DBA2A710816
:10147800A00061308A016321B2007108A0004130E8
:101488008A016321B400320834048A150A12031D44
:10149800BE2A7108A00067308A016321B200710872
:1014A800A00047308A016321B400320834048A1549
:1014B8000A12031DB52A7108A00077308A0163213A
:1014C800B2007108A00057308A016321B4003208C5
:1014D80034048A150A12031DB02A8A150A127D28B7
:1014E8000130D9008A018A276D08F000640070086D
:1014F8006E028A150A12031CAC2A6808EB00640005
:101508006B0869028A150A12031CA72A8A01B522E8
:1015180064005908003C8A150A12031D9C2A8A0196
:10152800CE226308D5008A0193268A150A12A22AB8
:101538008A01A726500888008A01F321EB0A8A1538
:101548000A12031D832AF00A8A150A12031D7A2A31
:10155800D9018A150A127D280230D9008A150A1283
:10156800C02A0330D9008A150A12C02AD9018A155F
:101578000A12C02A0130D9008A018A276808C800DF
:101588006908C7006D08CA006E08C9004708C50089
:101598004808C6004508A0004608A1004A08A3005C
:1015A80049088A0168218A150A12031D3F2B640025
:1015B8005908003C8A150A12031DFB2A8A01A7262E
:1015C8000730BA001030B8000730BB000830B90047
:1015D800A0308A01202046088A01202045088A0177
:1015E800202050088A011E200A308A012C2164001C
:1015F8005908013C8A150A12031D182B0730BA0036
:101608001030B8000730BB000830B900A0308A019C
:10161800202046088A01202045088A0120208A01C6
:101628000520D5008A01932664005908023C8A15D2
:101638000A12031D2B2B8A01A726450803178D00C4
:10164800031350088A011E210A308A012C216400E4
:101658005908033C8A150A12031D382B45088A01CC
:101668001621D5008A019326C50A0319C60A8A15C8
:101678000A12031DCE2AD9018A150A127D288A0169
:1016880023278A01E6278A01FE248A150A127D2863
:101698008A0123278A01E6278A01BF258A150A12AB
:1016A8007D288A0123278A01E6278A0185258A154C
:1016B8000A127D288A0123278A01E6278A01F12553
:1016C8008A150A127D288A018A278A0173278A01C6
:1016D8006C268A150A127D288A018A278A017327AF
:1016E8008A014D238A150A127D288A017327E80189
:1016F8007F30E900ED013F30EE008A016C268A1543
:101708000A127D288A018A278A015B248A150A120F
:101718007D288A150A127D280130E6008A01DF2615
:101728008A01ED278A01F921E6018A150A127D2826
:101738008A0136228A150A127D288A01DF268A0143
:10174800ED278A0173278A01B5228A01DB238A15CE
:101758000A127D288A01DF268A01ED278A01B5222F
:101768006B08F7008A01732764005508403C8A1506
:101778000A120319D82B8A01DB23640080306B021C
:101788008A150A12031CCA2B7708EB006400550857
:101798003B3C8A150A120319D32B8A011D238A019F
:1017A80073278A150A12B82B8A150A127D288A010E
:1017B800DF268A01ED276B08F7007008F8008A0118
:1017C800B5228A01732764005508403C8A150A121D
:1017D8000319042C8A01DB237708EB000830F00793
:1017E8006400403070028A150A12031CFD2B780829
:1017F800F0008A01B5228A0173278A150A12E72B9D
:101808008A150A127D288A0123278A01ED275208A2
:10181800D8008A01F9228A150A127D288A0123270D
:101828005008F4005108F3005208F6008A017327A3
:101838008A0135248A150A127D288A01232750082F
:10184800F6005108F5005208F4008A0173278A014E
:101858000F248A150A127D2863008A150A12302C73
:02400E00753DFE
:00000001FF
